:100000008EC095C094C093C092C091C090C08FC064
:100010008EC08DC08CC08BC08AC089C088C00006CD
:100020000C12181E242A30363C42484E545A606640
:100030006C72787E848A90969CA2A8AEB4BAC0C630
:10004000CCD2D8DEE4EAF0F6FFFFFFFFFFFFFFFFB0
:10005000FFFFFFFFFFFFFFFFFFFFFFFFFFFFFFFFB0
:10006000FFFFFFFFFFFFFFFFFFFFFFFFFFFFFFFFA0
:10007000FFFFFFFFFFFFFFFFFFFFFFFFFFFFFFFF90
:10008000FFFFFFFFFFFFFFFFFFFFFFFFFFFFFFFF80
:10009000FFFFFFFFFFFFFFFFFFFFFFFFFFFFFFF976
:1000A000F3EDE7E1DBD5CFC9C3BDB7B1ABA59F99F0
:1000B000938D87817B756F69635D57514B453F39E0
:1000C000332D27211B150F09000000000000000040
:1000D0000000000000000000000000000000000020
:1000E0000000000000000000000000000000000010
:1000F0000000000000000000000000000000000000
:1001000000000000000000000000000000000000EF
:1001100000000000000000000000000000001124AA
:100120001FBECFE5D2E0DEBFCDBF1AD0A1C068CFE1
:100130000F931F9300E010E0980106171707280798
:10014000390759F0E7E8F3E13197F1F700C0000013
:100150000F5F1F4F2F4F3F4FF0CF1F910F9108950B
:10016000F89480E886BD16BC80EE81BF88E087BB2E
:1001700080E090E001968F3F910511F480E090E0DF
:10018000582F482F4E6F20E8622F6423322F369568
:10019000C398662369F0232F0000000000000000D0
:1001A000000000000000000000000000C39A07C02B
:1001B00000000000C39A232F000000000000000090
:1001C0000000000000003111DFCF20E8622F64231F
:1001D000322F3695C398662369F0232F0000000064
:1001E000000000000000000000000000000000000F
:1001F000C39A07C000000000C39A232F000000002C
:10020000000000000000000000003111DFCF452F8A
:10021000406820E8522F5423322F3695C398552337
:1002200069F0232F00000000000000000000000023
:100230000000000000000000C39A07C0000000009A
:10024000C39A232F000000000000000000000000FF
:1002500000003111DFCFC398EFE4F3EC3197F1F7F1
:1002600000C00000C39AF6EAFA95F1F700C082CF09
:04027000F894FFCF30
:00000001FF
